:0600000002000E02001CCC
:10000B000200287581301200751200E612003B01C8
:10001B001AC0D0C0E0120128D0E0D0D032C0D0C07E
:10002B00E0D2B11200991200EBC2B1D0E0D0D032C5
:10003B00D2B175900075B0FF120060C2B175980017
:10004B00758A05758C0575890275881175B80274EA
:10005B008375A88322D2B2C21030B2FD20B2FD78D4
:10006B000C79FAD9FED8FAD21022A2B49202A2B518
:10007B009203A2B09206A2B392070200BCA2B59261
:10008B0002A2B09203A2B49206A2B3920722A2B428
:10009B009200A2B59201A2B09204A2B39205020003
:1000AB00BCA2B59200A2B09201A2B49204A2B392E8
:1000BB0005E520540F9000D693FCE520C4540F9017
:1000CB0000D693FDE5202323F5202200011000101C
:1000DB0000000101000010001001007A007B0022DB
:1000EB00EC2323239000F373210800000000000091
:1000FB000ABA10091A2108001ABA7F010AED232344
:10010B002390011073212700000000000000000B5A
:10011B00BB10091B2127001BBB7F010B22C2A97837
:10012B0014D8FEEAC4540FF59030B2FD780AD8FE0D
:10013B00EA540FF59020B2FD780AD8FEEBC4540FA9
:10014B00F59030B2FD780AD8FEEB540FF5907A009B
:07015B007B00C289D2A9223A
:00000001FF
